:102F00000C94AA170C94C5170C94C5170C94C517EC
:102F10000C94C5170C94C5170C94C5170C94C517C1
:102F20000C94C5170C94C5170C94C5170C94C517B1
:102F30000C94C5170C94C5170C94C5170C94C517A1
:102F40000C94C5170C94C5170C94C5170C94C51791
:102F50000C94C51711241FBECFE5D4E0DEBFCDBF52
:102F600010E0A0E6B0E0E0E6F7E302C005900D92C5
:102F7000A036B107D9F711E0A0E6B0E001C01D927C
:102F8000AE32B107E1F70C94021C0C948017F4C028
:102F90001FEF12BB1FEF18BB089512E011BB1AEA16
:102FA00017BB089512E011BB18E017BB0895552315
:102FB00012F0C19A01C0C1980895552312F0C1982A
:102FC00001C0C19A0895C79A13E11A95F1F7C798FD
:102FD0001AE01A95F1F7089509E109B908E10AB96B
:102FE00008955F9BFECF4CB108955D9BFECF4CB919
:102FF0000895C895002021F0402DF7DF3196F9CFD4
:103000000895C895002021F0402DEFDF3296F9CFCA
:103010000895C895002021F0501519F03296F9CF87
:1030200008940895C895002041F0501511F032968B
:10303000F9CF3196C895C02C8C2C0895C8950020E6
:1030400039F0501511F03296F9CF3196C895D02C41
:10305000089518E224E72A95F1F71A95D9F70A9509
:10306000C1F7089519D03D2F17D03C2F15D00895E2
:10307000312D12D0322D10D0332D0ED0342F0CD054
:103080000895312D09D0322D07D0332D05D003D02E
:10309000432FABDF0895332708E070E0331F10F4AF
:1030A000C59A01C0C598770FB69971608CDF0A95F3
:1030B000A9F7372F0895552322F030E2EDDF3D2F99
:1030C00003C03D2F41D03160E7DF3C2FE5DFE3DF78
:1030D000432F8BDF55234AF038E2DEDF3D2FDCDF64
:1030E0003C2FDADFD8DF432F80DF21960895552368
:1030F00022F030EAD1DF3D2F05C0573859F03D2F7F
:1031000023D03560C9DF3C2FC7DFC5DF432F6DDF1C
:10311000219608950F910F91A2C2552322F030EC11
:10312000BBDF3D2F05C0573861F03D2F0DD0366015
:10313000B3DF3C2FB1DF342FAFDF0AE08ADF219607
:1031400008950F910F918BC2330F330F330F18F483
:10315000573809F434600895C39808EC7ADF08EC16
:1031600078DF38ECC39A02E074DFC39801E071DFC6
:103170003A95C1F7C39A089500E1C02E8C2C50E215
:10318000AA24992405DF0EDF27DFE6DF2ADF4B3193
:10319000E9F3443579F425DF542FE5E4FBE1EE0F44
:1031A000FF1F40DF0FEFD02EE5E3FBE1EE0FFF1F27
:1031B00045DF58C2433531F4E9E7FBE1EE0FFF1F6D
:1031C00018DFE4CF463531F4E5E7FBE1EE0FFF1FF2
:1031D00010DFDCCF463731F4E7E7FBE1EE0FFF1FEE
:1031E00008DFD4CF443769F4E5E3FBE1EE0FFF1FBE
:1031F00008DFE5E4FBE1EE0FFF1F03DF40E0F5DE53
:10320000C5CF403719F443E5F0DEC0CF413619F49D
:1032100049E5EBDEBBCF493641F4EDE7FBE1EE0FCC
:10322000FF1FE7DE4AE0E1DE1DC2423639F449E520
:10323000DCDE40E0DADE40E2D8DEA8CF483719F421
:10324000D0DEC39A0FC2493719F4CBDEC3980AC245
:10325000E5E3FBE1EE0FFF1FDCDE38F4E5E4FBE124
:10326000EE0FFF1FD6DE08F4FAC1403509F028C082
:10327000C39893DEC7989BDE02E3EBDE9EDE02E39B
:10328000E8DE3CEA09DF33E507DF503280F0552302
:1032900072F020E200DF333561F030E0FDDE93DED6
:1032A0003CEAFADE33E5F8DE2A95A1F702C030E009
:1032B000F3DE552312F030E0EFDE04E0CADED2C1C7
:1032C0004336B9F48EDE30E4832F55231AF0E4DE62
:1032D0003D2F03C03D2F38DF3260DEDE3C2FDCDEC9
:1032E000342FDADE942F4C2E5D2E55230AF42196CE
:1032F0005DC1433491F475DE552372F038E4832FB9
:10330000CBDE3D2FC9DE3C2FC7DE342FC5DE942F28
:103310004C2E5D2E21964AC1A2C1423409F075C0DF
:1033200060DE442311F041E09AC15BDE413410F0CD
:1033300042E095C1642E742E54DEB42EBB27A0E665
:1033400050DE4D936A94E1F7BB27A0E621E0A22E60
:103350004B2D463449F0453411F043E080C14D9186
:10336000DCDE7A94E1F77EC1E5E4FBE1EE0FFF1FBE
:1033700050DE08F423C030E475DE3D918DDE38E484
:10338000832F70DE3D91932F4C2E5D2E85DE21968E
:103390007A9431F07A9421F0AA2069F38A9459F74B
:1033A000AA2009F45FC18A943CE476DE352D74DEF0
:1033B000342D72DE30E070DE8C2C23C15523DAF020
:1033C0009D919F3F41F030E4832F4CDE392F64DE26
:1033D0004C2E5D2EF2D07A949D919F3F41F038E4BF
:1033E000832F40DE392F58DE4C2E5D2EE6D02196FD
:1033F0007A9421F737C13D2FA7DE32604DDE3C2F96
:103400004BDE3D91932F48DEEFCF4235E1F455235B
:1034100022F038E241DE3D2F03C03D2F95DE3160C2
:103420003BDE3C2F39DE37DE432FDFDD55234AF00C
:1034300030E232DE3D2F30DE3C2F2EDE2CDE432FFD
:10344000D4DD2196A3CE4736B9F4CBDDB42FC9DD48
:10345000A42FC7DD463439F0453409F000C147DEFA
:103460001197E9F793CE27DE55231AF01297D9F773
:103470008DCE1197C1F78ACE413429F4B2DDD42F15
:10348000B0DDC42FEFC0443419F4ABDD46DEEAC032
:10349000443611F42CDE7ACE4C3421F488DD82DD02
:1034A000C39AE0C0453409F4F9CF453669F43CEAE3
:1034B000F3DD552312F030E8EFDD34E0EDDD30E0F0
:1034C000EBDD08E2C6DDCEC04C3649F48ADD3CEACD
:1034D000E3DD552382F0342F306EDEDD07C0463643
:1034E00099F47FDD3CEAD8DD30EAD6DD3327D4DD40
:1034F000342FD2DD06C0342F307E3760CDDD30E092
:10350000CBDD0AE0A6DDAEC0433771F455235AF097
:1035100020E3122E222422E0322EB3DD3A94B1DDD4
:103520003324AFDD33CE9BC04D3649F43CE4B4DDEB
:10353000352DB2DD342DB0DD30E0AEDD62C04A3372
:1035400051F44FDD142E4DDD242E4BDD342E99DD4C
:1035500002E37FDD87C04E3269F443DD142E41DD86
:10356000242E3FDD342E3DDD83DD472F3EDD02E39B
:1035700070DD78C0423711F438E503C0463421F4D9
:1035800030E58ADD33270AC04E3419F438E584DD8E
:1035900004C0413551F430E57FDD38E07DDD33276F
:1035A0007BDD79DD432F21DDF1CD59C0E5E4FBE181
:1035B000EE0FFF1F2EDD18F055C021E0922EDD200A
:1035C000D1F09D15C1F08F7080622227552322F023
:1035D000382F62DD352D03C0352DB6DD31605CDD61
:1035E000342D5ADD58DD552312F430789078391790
:1035F00021F02A9559F70AE02CDD992099F19924B8
:103600000895513499F05332D1F09F3F79F08F7083
:1036100080622227382F40DD352D3EDD342D3CDD04
:103620003ADD391729F02A9509F0F4CF02E311DDCC
:10363000AA2019F0772009F09ECEAA2413C080EFAB
:103640002227522E382F28DD352D26DD342D24DD7E
:1036500022DD317069F32A9549F3F4CFC6DC4FE3DC
:10366000C4DC94CD4DE0C1DC91CD1300207F287FD8
:1036700030FF34FF387F48FF4CFF51FF55FF56FFA6
:1036800068FF6CFF86FF87FF000001400440054093
:1036900006400740084009400E101A100F201B205A
:1036A00014201C201D40231031203320354037408A
:1036B00039403D403E4057103A203B204140434076
:1036C0004440454046405E10604061406240634077
:1036D0006440664069206A207240734074407540BF
:1036E000762077207840794000003338000032326D
:1036F000000041565220495350005665722E332E19
:1037000038622028415652313039204D6F64652C83
:103710002050617274206F662049736F4A7461672C
:103720004953507777772E666C6F70707973706F2E
:103730006E67656F6E6C696E652E636F6D202620F7
:103740007777772E6D696B726F636F6E74726F6CC3
:103750006C65722D70726F6A656B74652E6465009E
:1037A000033089F0053089F0073089F00B3089F05B
:1037B0000F3089F0073189F00F3189F00F3289F02D
:1037C0000F3589F011C003E00FC006E00DC008E01E
:1037D0000BC00CE009C000E107C009E105C002E22E
:0E37E00003C003E301C007E610BD09B9089558
:0238000001C005
:10380400C0E5D4E0DEBFCDBF11241A8219821D8227
:103814001C821F821E821886F89481E080935500D2
:1038240082E080935500809134008F7B8093340034
:1038340080913500806480933500809137008860E2
:10384400809337000E94621F80914E0081608093B4
:103854004E0080914E00846080934E0010924D0083
:1038640010924C001A86198689859A852AE2883F27
:10387400920741F48091380098E0892780933800BA
:103884001A86198689859A8501969A8789878091EF
:103894003300992780749070009799F480913800D0
:1038A40088608093380081E0809355001092550021
:1038B40010924E00809135008F7B809335000E94DA
:1038C400C71780912B0088233CF480912C008B87B0
:1038D4008B85833509F432C080914C0090914D0062
:1038E40038E98439930708F4BFCF8885813019F00B
:1038F40081E08887B9CF8091380088608093380050
:1039040081E0809355001092550010924E008091F2
:103914003300992780749070009741F080913500AE
:103924008F7B809335000E94721F9ECF809135005B
:103934008F7B809335000E94C71796CF8091380003
:1039440088608093380010924E000E940A1F0E94E3
:10395400261F8B838B81282F33273F872E878E85C5
:103964009F858635910509F4B1C02E853F8527359D
:1039740031050CF04DC08E859F858534910509F481
:103984002DC22E853F8526343105ECF48E859F8526
:103994008B31910509F42FC22E853F852C313105D9
:1039A4002CF48E859F85009791F22EC22E853F853B
:1039B4002134310509F497C08E859F8583349105A0
:1039C40009F453C121C22E853F852235310509F4FE
:1039D400D7C08E859F85833591056CF42E853F85F0
:1039E4002C34310509F4A0C08E859F85803591055E
:1039F40009F496C009C22E853F852335310509F4A3
:103A04005BC08E859F858435910509F466C0FCC131
:103A14002E853F852D36310509F479C18E859F8524
:103A24008E369105F4F42E853F852336310509F44D
:103A34000EC18E859F858436910534F42E853F858D
:103A440021363105A9F1E0C18E859F858436910523
:103A540009F478C02E853F852536310509F478C1EF
:103A6400D3C18E859F858437910549F12E853F8585
:103A74002537310564F48E859F8580379105A1F043
:103A84002E853F852337310509F452C0BDC18E858B
:103A94009F858837910509F48BC12E853F85293789
:103AA400310509F490C1B0C183E50E94431F4FCF93
:103AB40089E50E94431F4BCF0E940A1F48CF84E729
:103AC4000E94431F80E00E94431F41CF81E30E9474
:103AD400431F80E30E94431F3ACF0E94261F8DE0BC
:103AE4000E94431F34CF0E94261F9927182F0027B6
:103AF4000E94261F9927802B912B90932A01809353
:103B040029012091290130912A01C901820F931FB3
:103B140090932D0180932C018DE00E94431F17CFB9
:103B24008DE00E94431F13CF8DE00E94431F0FCFEF
:103B340082E00E94431F84E90E94431F8EE10E9499
:103B4400431F05CF8091290180933E008091290174
:103B540090912A01892F992780933F0080913C00FE
:103B6400992782709070009709F0F8CF80913C00FB
:103B7400816080933C0080913D000E94431FE7CE0A
:103B84008C819D81009791F120912C0130912D0120
:103B94008C819D812817390781F48DEB0E94431F86
:103BA40080E10E94431F80912C0190912D01029687
:103BB40090932D0180932C01CACE20912C01309139
:103BC4002D018E819F812817390781F489EB0E948A
:103BD400431F89E00E94431F80912C0190912D0185
:103BE400029690932D0180932C01B1CE80915700C1
:103BF400992781709070009709F0F8CF81E1809344
:103C04005700E89580912C0190912D0101969D8794
:103C14008C87EC85FD8584918B878B850E94431F5F
:103C240080912C0190912D019D878C87EC85FD85D9
:103C340084918B878B850E94431F80912C019091E6
:103C44002D01029690932D0180932C0180CE8091BA
:103C54003800877F809338000E94261F99279A8313
:103C640089838DE00E94431F72CE0E94261F9927EC
:103C7400382F222789819A81822B932B9A838983D7
:103C840089819A813DEB8031930751F48EE094E968
:103C94009A83898380912C0190912D019D838C833B
:103CA40089819A8129EB8930920751F480ED9BE157
:103CB4009A83898380912C0190912D019F838E8317
:103CC400809138008860809338008091570099274C
:103CD40081709070009709F0F8CF41E020912C0199
:103CE40030912D0189819A810C01F901409357008B
:103CF400E895112480912C0190912D0102969093C6
:103D04002D0180932C018DE00E94431F20CE8091D1
:103D1400290190912A0137E18038930720F08DE042
:103D24000E94431F14CE8091570099278170907090
:103D3400009709F0F8CF25E080912C0190912D0196
:103D4400FC0120935700E8958DE00E94431FFFCDAE
:103D540010922A01109229018091290190912A013F
:103D640027E181309207E0F423E0809129019091CA
:103D74002A01FC0120935700E89580915700992768
:103D840081709070009709F0F8CF8091290190918B
:103D94002A0180589F4F90932A0180932901DCCFF8
:103DA40081E180935700E8958DE00E94431FCFCDB9
:103DB4000E94261F80913800877F809338008DE011
:103DC4000E94431FC4CD0E94261F80913800886042
:103DD400809338008DE00E94431FB9CD88E190E0C4
:103DE40028E00FB6F894A89581BD0FBE21BD8DE0E3
:103DF4000E94431FACCD10922D0110922C01109201
:103E04002A0110922901A3CD8FE30E94431F9FCD65
:103E1400CF93DF93CDB7DEB781E40E94431F86E5DD
:103E24000E94431F82E50E94431F82E40E94431FB5
:103E34008FE40E94431F8FE40E94431F84E50E9485
:103E4400431FDF91CF910895CF93DF93CDB7DEB7B2
:103E540021970FB6F894DEBF0FBECDBF80912B0023
:103E640088230CF0FBCF80912C00898389819927CA
:103E740021960FB6F894DEBF0FBECDBFDF91CF9170
:103E84000895CF93DF93CDB7DEB721970FB6F8949B
:103E9400DEBF0FBECDBF898380912B00992780722E
:103EA4009070009709F4F8CF898180932C002196B3
:103EB4000FB6F894DEBF0FBECDBFDF91CF9108954A
:103EC400CF93DF93CDB7DEB789E18093290088E1F2
:103ED40080932A0086E880934000DF91CF91089573
:103EE400CF93DF93CDB7DEB7F0E0E0E00994DF9144
:043EF400CF910895CD
:0400000300002F00CA
:00000001FF
